:100000000C945B000C9483000C9483000C9483008C
:100010000C9483000C9483000C9483000C94830054
:100020000C9483000C9483000C9483000C94830044
:100030000C9483000C9483000C9483000C94830034
:100040000C94F4020C9483000C9475050C948300BA
:100050000C9483000C9483000C9483000C94830014
:100060000C9483000C948300000024272A000025B0
:10007000282B000023262904040404040404040299
:100080000202020202030303030303010204081035
:100090002040800102040810200102040810200002
:1000A0000000070002010000030406000000000039
:1000B000000000004C0111241FBECFEFD4E0DEBFD2
:1000C000CDBF11E0A0E0B1E0ECE3FCE002C00590A0
:1000D0000D92AA33B107D9F711E0AAE3B1E001C04C
:1000E0001D92A53DB107E1F710E0C6EBD0E004C0DA
:1000F0002297FE010E941806C43BD107C9F70E944F
:1001000045010C941C060C94000087E491E00E94C9
:100110005D01882359F087E491E00E945A018093A1
:100120004401682F87E491E00E946501089540E84A
:1001300055E260E070E087E491E00E94600164E6CF
:1001400070E080E090E00E945F0361E080911B011D
:100150000E94460461E080911D010E94460461E016
:1001600080911F010E94460460E08EE00E944604D8
:1001700060E08FE00E94460460E080E10E94460457
:1001800060E081E10E94460461E08EE00E94640428
:1001900061E08FE00E94640461E080E10E946404F9
:1001A00061E081E10E94640480913A010E94D403DD
:1001B000815092403CF080E190E090933D0180932B
:1001C0003C0104C010923D0110923C01809121013C
:1001D0000E94D403815092403CF080E290E09093E2
:1001E0003F0180933E0104C010923F0110923E01F6
:1001F000809123010E94D403815092403CF080E41E
:1002000090E0909341018093400104C0109241011D
:1002100010924001809125010E94D40381509240A8
:100220003CF080E890E0909343018093420104C049
:10023000109243011092420180913E0190913F0142
:1002400020913C0130913D01820F931F209140018C
:1002500030914101820F931F20914201309143015F
:10026000820F931F909346018093450160E071E0F7
:1002700087E491E00E94750160914501709146010B
:1002800087E491E00E94C40208950E9497030E94AF
:1002900097000E948500FDCF87E391E0909348018D
:1002A000809347010895862F0E94340508950E9487
:1002B0006C0508950E944D0508950E943C0508951F
:1002C000CB01BA010E94FB040895DC01ED91FC9181
:1002D0000190F081E02D09950895DC01ED91FC91EC
:1002E0000190F081E02D099508950F931F93CF930E
:1002F000DF938C01EB0109C02196D801ED91FC91AF
:100300000190F081E02DC801099568816623A1F76D
:10031000DF91CF911F910F9108950F931F938C013F
:10032000DC01ED91FC910190F081E02D6DE00995EB
:10033000D801ED91FC910190F081E02D6AE0C801B7
:1003400009951F910F9108950F931F938C01DC0164
:10035000ED91FC910190F081E02D0995C8010E947A
:100360008D011F910F9108950F931F938C010E948F
:100370007501C8010E948D011F910F9108950F937F
:100380001F938C01DC01ED91FC910190F081E02D37
:100390000995C8010E948D011F910F9108952F9218
:1003A0003F924F925F926F927F928F929F92AF9205
:1003B000BF92CF92DF92EF92FF920F931F93DF9342
:1003C000CF93CDB7DEB7A0970FB6F894DEBF0FBEC0
:1003D000CDBF1C016A017B01411551056105710505
:1003E00049F4DC01ED91FC910190F081E02D60E396
:1003F000099554C0882499245401422E552466241A
:10040000772401E010E00C0F1D1F080D191DC70116
:10041000B601A30192010E94C505F801608308940A
:10042000811C911CA11CB11CC701B601A301920142
:100430000E94C505C901DA016C017D01C114D10416
:10044000E104F104F1F681E0E82EF12CEC0EFD1E42
:10045000E80CF91C3E010894611C711CD501C40113
:100460000197A109B1096C01C818D90814C0F60197
:10047000EE0DFF1D60816A3010F4605D01C0695CA3
:10048000D101ED91FC910190F081E02DC101099520
:100490000894E108F1086E147F0449F7A0960FB69E
:1004A000F894DEBF0FBECDBFCF91DF911F910F91AA
:1004B000FF90EF90DF90CF90BF90AF909F908F9084
:1004C0007F906F905F904F903F902F9008952AE01B
:1004D0000E94CF0108950F931F938C010E94670221
:1004E000C8010E948D011F910F910895AB0160E03A
:1004F00070E00E94670208950F931F938C01AB0177
:1005000060E070E00E946702C8010E948D011F91A7
:100510000F910895EF92FF920F931F93CF93DF9364
:10052000EC017A018B0177FF0FC0E881F98101901E
:10053000F081E02D6DE2099510950095F094E0941E
:10054000E11CF11C011D111D2AE0B801A701CE011B
:100550000E94CF01DF91CF911F910F91FF90EF90FB
:1005600008950F931F938C010E948A02C8010E9474
:100570008D011F910F910895AB01662757FD60957E
:10058000762F0E948A0208950F931F938C01AB016E
:10059000662757FD6095762F0E948A02C8010E9447
:1005A0008D011F910F910895DC012115310541F452
:1005B000ED91FC910190F081E02D642F0995089553
:1005C0002A30310519F40E948A0208950E94CF0151
:1005D00008950F931F938C010E94D402C8010E94BA
:1005E0008D011F910F9108951F920F920FB60F92D8
:1005F00011242F938F939F93AF93BF9380914901C1
:1006000090914A01A0914B01B0914C018050904CC7
:10061000AF4FBF4F8093490190934A01A0934B0184
:10062000B0934C0127C08091490190914A01A0915B
:100630004B01B0914C0180589E43A040B040809344
:10064000490190934A01A0934B01B0934C018091D2
:100650004D0190914E01A0914F01B0915001019632
:10066000A11DB11D80934D0190934E01A0934F01A8
:10067000B09350018091490190914A01A0914B01A2
:10068000B0914C0181589E43A040B04060F6BF91AC
:10069000AF919F918F912F910F900FBE0F901F9050
:1006A00018958FB7F89420914D0130914E014091EB
:1006B0004F01509150018FBFB901CA010895EF92C7
:1006C000FF920F931F937B018C018FB7F894409199
:1006D0004D0150914E0160914F01709150018FBFBB
:1006E0002FB7F89480914D0190914E01A0914F0148
:1006F000B09150012FBF841B950BA60BB70B8E1525
:100700009F05A007B10760F31F910F91FF90EF9035
:100710000895019759F0FC01EE0FFF1FEE0FFF1F28
:1007200032978FB7F8943197F1F78FBF0895789487
:1007300084B5826084BD84B5816084BD85B58260E6
:1007400085BD85B5816085BDEEE6F0E08081816084
:100750008083E1E8F0E08081826080838081816035
:100760008083E0E8F0E0808181608083E1EBF0E06D
:10077000808184608083E0EBF0E080818160808311
:10078000EAE7F0E0808184608083808182608083FA
:100790008081816080838081806880831092C10025
:1007A00008958093390108958F7090913901929541
:1007B000990F990F907C982B90937C0080917A00F0
:1007C000806480937A0080917A0086FDFCCF20912E
:1007D000780040917900942F80E030E0282B392B6D
:1007E000C90108951F93CF93DF93182FEB0161E0A8
:1007F0000E944604E12FF0E0E156FF4F84918330E0
:1008000051F480918000806880938000D0938900AB
:10081000C093880037C0843051F48091800080629A
:1008200080938000D0938B00C0938A002BC08130CE
:1008300029F484B5806884BDC7BD24C0823029F402
:1008400084B5806284BDC8BD1DC0863041F48091EE
:10085000B00080688093B000C093B30013C08730AD
:1008600041F48091B00080628093B000C093B400E6
:1008700009C0C038D10514F460E001C061E0812FE7
:100880000E946404DF91CF911F910895282F30E0DA
:10089000C90185579F4FFC01949129583F4FF90199
:1008A0008491882381F0E82FF0E0E859FF4FE4912C
:1008B000F0E0662329F48081909589238083089550
:1008C0008081892B80830895482F50E0CA0181568A
:1008D0009F4FFC012491CA0185579F4FFC019491C1
:1008E00049585F4FFA0134913323C1F1222331F18A
:1008F000233021F4809180008F7705C0243031F4BB
:10090000809180008F7D8093800018C0213019F481
:1009100084B58F7704C0223021F484B58F7D84BDE7
:100920000DC0263021F48091B0008F7705C02730AC
:1009300029F48091B0008F7D8093B000E32FF0E028
:10094000E359FF4FE491F0E0662329F4808190950C
:100950008923808308958081892B80830895482F7F
:1009600050E0CA0181569F4FFC012491CA0185576E
:100970009F4FFC01949149585F4FFA013491332302
:1009800019F420E030E035C0222331F1233021F486
:10099000809180008F7705C0243031F480918000F1
:1009A0008F7D8093800018C0213019F484B58F7733
:1009B00004C0223021F484B58F7D84BD0DC0263063
:1009C00021F48091B0008F7705C0273029F4809101
:1009D000B0008F7D8093B000E32FF0E0EE58FF4F22
:1009E000E491F0E0808120E030E0892311F021E003
:1009F00030E0C9010895EF92FF920F931F937B019E
:100A00008C0122E030E040E050E00E94E705205CED
:100A10003D4B404F5F4FCA01B901A80197010E94A9
:100A2000E705C901DA010197A109B109292F3A2F78
:100A30004B2F552747FD5A950196A11DB11D2093B7
:100A4000C50081508093C400E1ECF0E080818061BA
:100A500080838081886080838081806880831F910B
:100A60000F91FF90EF900895982F8091C00085FF1F
:100A7000FCCF9093C600089580915101909152014E
:100A800080589F4F2091530130915401821B930B4A
:100A900060E870E00E94B2050895409153015091C2
:100AA000540180915101909152018417950719F4D6
:100AB0002FEF3FEF0FC0FA01EB5AFE4F2081CA0122
:100AC000019660E870E00E94B20590935401809313
:100AD000530130E0C9010895809153019091540170
:100AE000909352018093510108951F920F920FB677
:100AF0000F9211242F933F934F935F936F937F93A4
:100B00008F939F93AF93BF93EF93FF934091C60052
:100B1000E0915101F0915201CF01019660E870E03F
:100B20000E94B2059C0180915301909154012817B5
:100B3000390739F0EB5AFE4F40833093520120932E
:100B40005101FF91EF91BF91AF919F918F917F9153
:100B50006F915F914F913F912F910F900FBE0F902A
:100B60001F90189597FB092E07260AD077FD04D011
:100B700049D006D000201AF4709561957F4F0895F2
:100B8000F6F7909581959F4F0895A1E21A2EAA1B22
:100B9000BB1BFD010DC0AA1FBB1FEE1FFF1FA2172D
:100BA000B307E407F50720F0A21BB30BE40BF50B2A
:100BB000661F771F881F991F1A9469F760957095B3
:100BC000809590959B01AC01BD01CF01089597FBE5
:100BD000092E05260ED057FD04D0D7DF0AD0001C01
:100BE00038F450954095309521953F4F4F4F5F4FCA
:100BF0000895F6F790958095709561957F4F8F4F8A
:100C00009F4F0895AA1BBB1B51E107C0AA1FBB1F22
:100C1000A617B70710F0A61BB70B881F991F5A9588
:100C2000A9F780959095BC01CD010895EE0FFF1FA7
:0C0C30000590F491E02D0994F894FFCF9A
:100C3C00486F6C612C20736F7920656C20726F6229
:100C4C006F74206E756D65726F2000060008000BC6
:100C5C000001000200030009000A00020003000565
:0A0C6C000004000000000053010125
:00000001FF
